:100000000C942A000C9445000C9445000C94450077
:100010000C9445000C9445000C9445000C9445004C
:100020000C9445000C9445000C9445000C9445003C
:100030000C9445000C9445000C9445000C9445002C
:100040000C9445000C9445000C9445000C9445001C
:100050000C94450011241FBECFE5D8E0DEBFCDBF14
:1000600010E0A0E6B0E0ECEDF8E002C005900D92E3
:10007000A439B107D9F710E0A4E9B0E001C01D929E
:10008000A439B107E1F70C94EC030C94000000973D
:1000900011F00197F1F70895DD9ADD9808951BBAE4
:1000A0000E944C0081E08BBB0E944C0088EE93E0E4
:1000B0000E94470008951BBA0E944C0082E08BBB4F
:1000C0000E944C0088EE93E00E94470008950F9331
:1000D0001F93CF93182FC62F042F1BBA0E944C00DA
:1000E00088E0113029F0C13031F0013041F406C010
:1000F0008CE0C130D1F78260013009F481608BBBA4
:100100000E944C0084E690E00E944700CF911F912E
:100110000F9108951F93182F82958F7088608BBB65
:100120000E944C001F701BBB0E944C0084E690E0B4
:100130000E9447001F9108951F93182F82958F707A
:1001400080618BBB0E944C00812F8F7080618BBBC4
:100150000E944C0084E690E00E9447001F910895A1
:10016000CF93DF93EC018881882361F089910E940D
:100170009C008881882331F089910E949C008881AD
:100180008823A1F7DF91CF9108951F93CF93182F64
:10019000C0E802C080E304C0812F8C23D9F381E33F
:1001A0000E949C00C695C1F7CF911F910895CF93EF
:1001B000982F82958F70805D8A3308F0895F9F70D9
:1001C000C92FC05DCA3308F0C95F0E949C008C2F04
:1001D0000E949C00CF9108950F931F93CF93DF93BC
:1001E000EC0184369105D8F46AE070E00E9438048E
:1001F0008B01862F805D0E949C00C801880F991F8B
:10020000880F991F880F991F800F911F800F911FD2
:10021000C81BD90B8C2F805D0E949C0004C080E617
:1002200090E00E94B000DF91CF911F910F9108954F
:10023000EF92FF920F931F93CF93DF93EC0183E034
:10024000C83ED80788F544E6E42EF12CCE01B7016C
:100250000E9438048B01862F805D0E949C000E9DB9
:10026000C0010F9D900D1E9D900D1124C81BD90B30
:10027000CE016AE070E00E9438048B01862F805D19
:100280000E949C00C801880F991F880F991F880F32
:10029000991F800F911F800F911FC81BD90B8C2FA6
:1002A000805D0E949C0004C080E690E00E94B00047
:1002B000DF91CF911F910F91FF90EF900895CF9212
:1002C000DF92EF92FF920F931F937C01E0E1CE2E1D
:1002D000E7E2DE2EB6010E9438048B01862F805D96
:1002E0000E949C000C9DC0010D9D900D1C9D900DC9
:1002F0001124E81AF90A78EEC72E73E0D72EC70149
:10030000B6010E9438048B01862F805D0E949C00FC
:100310000C9DC0010D9D900D1C9D900D1124E81A9F
:10032000F90A64E6C62ED12CC701B6010E94380432
:100330008B01862F805D0E949C000C9DC0010D9D4D
:10034000900D1C9D900D1124E81AF90AC7016AE06E
:1003500070E00E9438048B01862F805D0E949C0013
:10036000C801880F991F880F991F880F991F800F48
:10037000911F800F911FE81AF90A8E2D805D0E944F
:100380009C001F910F91FF90EF90DF90CF90089508
:10039000AF92BF92CF92DF92EF92FF920F931F9393
:1003A000CF93DF937B018C01A12C9AECB92E9AE9B3
:1003B000C92E9BE3D92EC801B701A60195010E9461
:1003C0004C04E901822F805D0E949C00CE01AA2787
:1003D000BB27BC01CD01A60195010E941904DC01D7
:1003E000CB01E81AF90A0A0B1B0BA12C81EEB82EDF
:1003F00085EFC82E85E0D82EC801B701A60195016A
:100400000E944C04E901822F805D0E949C00CE0175
:10041000AA27BB27BC01CD01A60195010E941904A2
:10042000DC01CB01E81AF90A0A0B1B0BC0E8AC2E61
:10043000C6E9BC2EC8E9CC2ED12CC801B701A60153
:1004400095010E944C04E901822F805D0E949C006E
:10045000CE01AA27BB27BC01CD01A60195010E94B0
:100460001904DC01CB01E81AF90A0A0B1B0BB0E4F2
:10047000AB2EB2E4BB2EBFE0CB2ED12CC801B7010E
:10048000A60195010E944C04E901822F805D0E9423
:100490009C00CE01AA27BB27BC01CD01A601950176
:1004A0000E941904DC01CB01E81AF90A0A0B1B0BA4
:1004B000A0EAAA2EA6E8BA2EA1E0CA2ED12CC80125
:1004C000B701A60195010E944C04E901822F805DCD
:1004D0000E949C00CE01AA27BB27BC01CD01A6012A
:1004E00095010E941904DC01CB01E81AF90A0A0BF4
:1004F0001B0BC801B70120E137E240E050E00E9449
:100500004C04E901822F805D0E949C0080E197E20B
:10051000C89F9001C99F300DD89F300D1124C9018B
:10052000AA27BB27E81AF90A0A0B1B0BC801B70157
:1005300028EE33E040E050E00E944C04E901822FB5
:10054000805D0E949C0088EE93E0C89F9001C99F47
:10055000300DD89F300D1124C901AA27BB27E81AF6
:10056000F90A0A0B1B0BC801B70124E630E040E092
:1005700050E00E944C04E901822F805D0E949C00A3
:1005800084E690E0C89F9001C99F300DD89F300D40
:100590001124C901AA27BB27E81AF90A0A0B1B0B69
:1005A000C801B7012AE030E040E050E00E944C046E
:1005B000E901822F805D0E949C00CE01880F991F67
:1005C000880F991F880F991F8C0F9D1F8C0F9D1FDF
:1005D000AA27BB27E81AF90A0A0B1B0B8E2D805D90
:1005E0000E949C00DF91CF911F910F91FF90EF909F
:1005F000DF90CF90BF90AF9008951F938FEF8ABB8D
:1006000080E197E20E94470013E01BBB0E944C0070
:1006100084EF91E00E9447001BBB0E944C0084E6DF
:1006200090E00E9447001BBB0E944C0084E690E0D3
:100630000E94470012E01BBB0E944C0084E690E041
:100640000E9447001BBB0E944C0088E08BBB0E94AD
:100650004C0084E690E00E9447001BBA0E944C00C8
:100660008FE08BBB0E944C0084E690E00E94470024
:100670001BBA0E944C0086E08BBB0E944C0084E6B3
:1006800090E00E9447000E944F001F9108958F92B2
:100690009F92AF92BF92CF92DF92EF92FF920F9311
:1006A0001F93CF93DF93CDB7DEB75FE0A52EB12CBC
:1006B000AC0EBD1EF501C190D1905F01F601819194
:1006C0006F01853251F0882309F46AC00E949C00B2
:1006D000F60181916F018532B1F791916F01892FF8
:1006E000292F332727FD30952436310509F449C0D9
:1006F0002536310564F42336310541F7F50122E052
:1007000030E0A20EB31E80810E949C00E1CF28370A
:100710003105E1F620E1E22EF12C4701F50122E05E
:1007200030E0A20EB31E008111819436B9F0C801E9
:10073000B7010E943804FB01EC59FF4F80810E94F1
:100740009C00C801B7010E9438048C01C701B401A4
:100750000E9438047B01672B51F7B0CF17FD19C0F9
:1007600032E0E316F10418F30E151F0500F7C70178
:100770006AE070E00E9438047B0162307105A0F7E6
:10078000D6CF4AE0842E912C30E1E32E37E2F32ECF
:10079000C5CF109501951F4F8DE20E949C00E0CFC0
:1007A00080E090E0DF91CF911F910F91FF90EF904B
:1007B000DF90CF90BF90AF909F908F90089540E0D2
:1007C00050E006C023E6225327FFFDCF4F5F5F4F67
:1007D00048175907B8F30895CFE5D8E0DEBFCDBF7D
:1007E0000E94FD0240E0642F81E00E94670085E7DF
:1007F00090E00E94B00080E40E948A008AEA90E0C3
:100800009F938F938FED90E09F938F938AEE9FEF4E
:100810009F938F9386E890E09F938F930E94470366
:100820008DB79EB708960FB6F8949EBF0FBE8DBFCA
:10083000FFCF629FD001739FF001829FE00DF11DF9
:10084000649FE00DF11D929FF00D839FF00D749F4A
:10085000F00D659FF00D9927729FB00DE11DF91FF6
:10086000639FB00DE11DF91FBD01CF011124089553
:10087000AA1BBB1B51E107C0AA1FBB1FA617B707C6
:1008800010F0A61BB70B881F991F5A95A9F78095E2
:100890009095BC01CD010895A1E21A2EAA1BBB1BA5
:1008A000FD010DC0AA1FBB1FEE1FFF1FA217B3073C
:1008B000E407F50720F0A21BB30BE40BF50B661F52
:1008C000771F881F991F1A9469F760957095809516
:0C08D00090959B01AC01BD01CF01089583
:1008DC004572720030313233343536373839414253
:1008EC0043444546002048656C6C6F2066726F6D02
:1008FC0020415652200054656D703D25642563439C
:04090C00202578002A
:00000001FF
